:020000040000FA
:06000000A4EF19F012004C
:0600080004EF08F01200F5
:060018000CEF08F01200DD
:06100000A4EF19F012003C
:021006001200D6
:0610080091EF10F0120050
:061018009AEF10F0120037
:02101E000100CF
:0C10200064330000C10000000C00000060
:04102C00D9CFE6FF33
:10103000E1CFD9FFE6520F015F6B626A160E616E57
:101040009F0E5B6F7B0E606E648C5C6B040EE66EB5
:10105000E66AE66A540EE66E0F0EE66E7AEC19F05A
:10106000146E050EE15E1450649CDF6ADF50146E4E
:10107000156A140E145C000E155810E2DF50040DB2
:10108000F3CFE9FFF4CFEAFF000EE926020EEA22D1
:10109000EE6AEE6AEE6AEE6ADF2AE8D70F01160EF4
:1010A000536F62A602D06296FCD700017F6B846BFF
:1010B000856B866B6498080E716F020E726F616BA0
:1010C000606BE552E552E7CFD9FF1200D9CFE6FFBA
:1010D000E1CFD9FFE6520001605117E106D0646A02
:1010E000606A0001606BA194AAD0646A606A160EFF
:1010F000616E0F019F0E5B6F7B0E606E64B602D057
:101100006486FCD70001010E606F600508E164BAD7
:1011100006D0626A606A60806088020E606F62500A
:10112000040B05E06050040B02E06294B9D864A29D
:1011300002D0A19484D06250010B12E06050010BE8
:101140000FE074DF0001040E606F0201500E026FA9
:10115000020E036F080E016F006B8C0E001362907D
:101160006250100B05E06050100B02E087D86298C7
:101170006250400B13E06050400B10E0010EE66E31
:10118000E66A000EE66EE66A730EE66EE66AF3EC59
:1011900016F0146E060EE15E1450629C6250200B35
:1011A00004E06050200B01E04FD86250020B14E0C5
:1011B0006050020B11E0010EE66EE66A000EE66E6C
:1011C000E66AE6687F0EE66EF3EC16F0146E060E25
:1011D000E15E14500F015F6B040E0001E76E6019B1
:1011E000E8AE02D0E73402D0E750605D02E2A1949D
:1011F00026D060A623D0DF6A040EDF5C1FE262A661
:101200001AD063CF8CF06296780E00018C1502E143
:101210005CD810D0000EE66EE66A8C0EE66E000E0C
:10122000E66E720EE66EE66AF3EC16F0146E060ECB
:10123000E15E145001D002D0DF2ADED7A194E5523E
:10124000E552E7CFD9FF12000F0153A115D063C0BB
:10125000E9FF64C0EAFFEF5080080DE171C0E9FFCB
:1012600072C0EAFFEF50840806E163C0E9FF64C082
:10127000EAFF8C0EEF6E5391629A120060846298BE
:101280006482000EE66EE66AE66EE66A750EE66E4B
:10129000E66AF3EC16F0146E060EE15E14501200CE
:1012A000000EE66EE66AE66EE66A740EE66EE66AC2
:1012B000F3EC16F0146E060EE15E14506492609426
:1012C00062A402D06294FCD71200D9CFE6FFE1CF2E
:1012D000D9FFE652FD0E00018C155AE17E0E8C15E9
:1012E000E8407F0B040DF3CF63F0F4CF64F0000E01
:1012F0006327020E642363C065F064C066F0657501
:1013000063C0E9FF64C0EAFFEF503C0BE842E842EB
:101310000D083CE163C0E9FF64C0EAFF020EE92664
:10132000000EEA22EECF14F0EFCF15F0580E14188D
:1013300002E1020E151828E163C0E9FF64C0EAFF6C
:10134000020EE926000EEA22500EEE6E020EED6E3F
:10135000DF6ADF50146E156A080E145C000E155813
:1013600013E2DF50EA6A580FE96E020EEA22EF50EC
:10137000E66EDF50EA6A500FE96E020EEA22E5528D
:10138000E750EF6EDF2AE5D70DD801D02ED805D073
:10139000FD0E8C15040801E14ED8E552E552E7CF69
:1013A000D9FF120071C0E9FF72C0EAFFEF50800B55
:1013B00005E071C0E9FF72C0EAFFEF6A00017B6BD4
:1013C0007C6B806B816B7F6BB9D8000EE66EE66A32
:1013D000E66EE66A030EE66EE66AF3EC16F0146E4D
:1013E000060EE15E145049EF0CF0020E00017C5D28
:1013F00002E1AFDB1FD06FD800018D511AE165C04B
:10140000E9FF66C0EAFFEE52080EEF6E65C0E9FF25
:1014100066C0EAFF020EE926000EEA22500EEE6ECA
:10142000020EED6E65C0E9FF66C0EAFF8C0EEF6E3E
:1014300001D08D6B1200D9CFE6FFE1CFD9FFE65284
:1014400071C0E9FF72C0EAFFEF50400B01E0010EEE
:10145000DF6E00017175080E605D0DE152C25CFF28
:101460000F015C51000804E20001100E606F03D010
:101470000001040E606F7C0528E171C0E9FF72C0B5
:10148000EAFF020EE926000EEA22580EEE6E020E68
:10149000ED6ED4DA020E00017B5D07E171C0E9FF59
:1014A00072C0EAFF840EEF6E0FD0DF5007E171C00B
:1014B000E9FF72C0EAFFC80EEF6E06D071C0E9FF07
:1014C00072C0EAFF880EEF6E01D005D8E552E552F2
:1014D000E7CFD9FF1200D9CFE6FFE1CFD9FF020E47
:1014E000E12600017C6B71C0E9FF72C0EAFFEF6A80
:1014F000040E7119146E72C015F014C0DEFF15C011
:10150000DDFFDECFE9FFDDCFEAFFEF6A84AF0CD06D
:101510008751881107E005D088C0FAFF0001875184
:10152000F96EFADF0001849F020EE15C02E2E16ADB
:10153000E552E16EE552E7CFD9FF120002015051AA
:10154000600BE842E842E842E842E842000901E074
:1015500058D051510C0A54E00B0A43E00C0A35E014
:10156000010A26E00B0A22E0020A20E0030A1CE03E
:10157000080A10E0010A0CE00F0A08E0030A01E083
:101580003FD000017F8F080E606F3BD0C7D839D0A5
:101590007EDB37D00001610E7D6F000E7E6F7F8194
:1015A000010E806F7F8F2DD013D92BD02BD829D04F
:1015B000545100017D6F7E6B620E7D27000E7E23ED
:1015C0007F81010E806F7F8F1CD000017F8F020111
:1015D0005451EA6A620FE96E000EEA2252C2EFFF2E
:1015E00010D0000EE66EE66AE66EE66A020EE66E61
:1015F000E66AF3EC16F0146E060EE15E145001D0AC
:1016000000D01200D9CFE6FFE1CFD9FF040EE126CA
:101610000201520510E150511F0B00090CE10001BD
:101620007F8F030E0201515D04E10001010E8B6FFB
:1016300002D000018B6B0201525166E150511F0B29
:10164000020862E154510F0B00095EE000017F8F38
:10165000020154BF10D054510F0BE96EEA6AD890C2
:10166000E936EA36670EE926000EEA22EECFDEFF03
:10167000EDCFDDFF0FD054510F0BE96EEA6AD89021
:10168000E936EA36710EE926000EEA22EECFDEFFD9
:10169000EDCFDDFF030E515D07E1DECFE9FFDDCFCA
:1016A000EAFF840EEF6E30D054510F0B156A530FC2
:1016B000146E0F0E1522020E14C0DBFF030E15C0B0
:1016C000DBFF020EDBCFE9FF030EDBCFEAFFEF907B
:1016D00054AF0DD0DECFE9FFDDCFEAFFEF6ADF7454
:1016E000DECFE9FFDDCFEAFF400EEF6E0DD0DECF9B
:1016F000E9FFDDCFEAFF880EEF6EDF74DECFE9FF92
:10170000DDCFEAFFC80EEF6E040EE15C02E2E16A93
:10171000E552E16EE552E7CFD9FF1200800E0201DB
:10172000505D55E10001C00E7F6F02015351030A65
:101730002EE0010A0EE0030A03E000017F6B47D0B0
:1017400000017C0E7D6F2E0E7E6F120E806F816BFE
:101750003ED05251F66EF76AD890F636F736290E1B
:10176000F626300EF7220900F5CF7DF00A00F5CFFE
:101770007EF0020E0001F76A7D25F66E7E51F7229B
:101780000900F5CF80F00A00F5CF81F020D0030EDC
:10179000525D1AE25251F66EF76AD890F636F73675
:1017A0002B0EF626300EF7220900F5CF7DF00A0049
:1017B000F5CF7EF07DC0F6FF7EC0F7FF0800F55044
:1017C0000001806F816B02D000017F6B00D012009E
:1017D000D9CFE6FFE1CFD9FF020EE1260201586B17
:1017E000596B50511F0B020A12E0030A0DE0010A67
:1017F00001E03BD000017F8F0201588100018B0581
:1018000002E10201588331D000017F8F2ED0000108
:101810007F8F020154BF10D054510F0BE96EEA6A5A
:10182000D890E936EA36670EE926000EEA22EECFB6
:10183000DEFFEDCFDDFF0FD054510F0BE96EEA6AEA
:10184000D890E936EA36710EE926000EEA22EECF8C
:10185000DEFFEDCFDDFFDECFE9FFDDCFEAFFEF50AA
:10186000040B02E0010E586F00D000017FAF07D0DB
:10187000580E7D6F020E7E6F7F81020E806F020E0A
:10188000E15C02E2E16AE552E16EE552E7CFD9FFA1
:101890001200649800017FBF4AD084AF28D0020EA6
:1018A0007C6F71C0E9FF72C0EAFFEE52EF6A71C04F
:1018B000E9FF72C0EAFFC80EEF6E65C0E9FF66C0BF
:1018C000EAFFEE52080EEF6E65C0E9FF66C0EAFF60
:1018D000020EE926000EEA22580EEE6E020EED6EA2
:1018E00065C0E9FF66C0EAFFC80EEF6E1FD065C095
:1018F000E9FF66C0EAFFEE52080EEF6E65C0E9FF31
:1019000066C0EAFF020EE926000EEA22500EEE6ED5
:10191000020EED6E65C0E9FF66C0EAFF8C0EEF6E49
:1019200071C0E9FF72C0EAFF840EEF6E86D084BFFB
:1019300084D0020150AF59D0000180510201565DA0
:10194000000181510201575904E256C280F057C28A
:1019500081F074D80001010E7C6F65C0E9FF66C09C
:10196000EAFFEE52080EEF6E65C0E9FF66C0EAFFBF
:10197000020EE926000EEA22500EEE6E020EED6E09
:1019800065C0E9FF66C0EAFF800EEF6E8D6B63C035
:10199000E9FF64C0EAFFEE52080EEF6E63C0E9FF94
:1019A00064C0EAFF020EE926000EEA22500EEE6E37
:1019B000020EED6E63C0E9FF64C0EAFF840EEF6EB5
:1019C000010E8D6F71C0E9FF72C0EAFF020EE926B9
:1019D000000EEA22580EEE6E020EED6E71C0E9FFA7
:1019E00072C0EAFFC80EEF6E28D00001020E7C6FB5
:1019F00071C0E9FF72C0EAFFEE52EF6A71C0E9FF01
:101A000072C0EAFFC80EEF6E65C0E9FF66C0EAFF6C
:101A1000EE52080EEF6E65C0E9FF66C0EAFF020EE7
:101A2000E926000EEA22580EEE6E020EED6E65C03B
:101A3000E9FF66C0EAFFC80EEF6E1200D9CFE6FFDD
:101A4000E1CFD9FF020EE1260001080E805D000EF5
:101A500081590EE280C0DEFF81C0DDFF7B5103E1D2
:101A6000010E7B6F04D07B0502E1020E7B6F03D079
:101A7000080EDE6EDD6A71C0E9FF72C0EAFFEF9208
:101A800071C0E9FF72C0EAFFEF9071C0E9FF72C058
:101A9000EAFF010EDB50EF1271C0E9FF72C0EAFFEE
:101AA000EE52DFCFEFFF000EDB50805F010EDB5008
:101AB000815B580E896F020E8A6F7FB121D0D9CF1A
:101AC000E9FFDACFEAFFEE50ED1019E07DC0F6FF36
:101AD0007EC0F7FF7D2B000E7E230800F550E66EDA
:101AE00089C0E9FF8AC0EAFF892B000E8A23E552EC
:101AF000E750EF6EDF06010E01E2DB06E0D71FD0F4
:101B0000D9CFE9FFDACFEAFFEE50ED1018E07DC043
:101B1000E9FF7EC0EAFF7D2B000E7E23EF50E66ECC
:101B200089C0E9FF8AC0EAFF892B000E8A23E552AB
:101B3000E750EF6EDF06010E01E2DB06E1D7020E91
:101B4000E15C02E2E16AE552E16EE552E7CFD9FFDE
:101B50001200D9CFE6FFE1CFD9FF020EE12663C024
:101B6000E9FF64C0EAFFEE52EFCFDFFFDFCF14F0F2
:101B700014500001855D000E865903E285C0DFFF29
:101B800009D0DF50146E156A1450855D856F1550AD
:101B90008659866F010EDB6ADF50F36E010EDBCFD4
:101BA000F4FFF350F45C16E2010EDB50EA6A580FC2
:101BB000E96E020EEA22EF50E66E82C0E9FF83C0B2
:101BC000EAFF822B000E8323E552E750EF6E010EF1
:101BD000DB2AE2D7000ED8808555000E865528E214
:101BE00065C0E9FF66C0EAFFEE52080EEF6E65C001
:101BF000E9FF66C0EAFF020EE926000EEA22580E4F
:101C0000EE6E020EED6E63C0E9FF64C0EAFFEF50B6
:101C1000400B07E165C0E9FF66C0EAFFC80EEF6E42
:101C200006D065C0E9FF66C0EAFF880EEF6E25D0DA
:101C300065C0E9FF66C0EAFFEE52080EEF6E65C0B0
:101C4000E9FF66C0EAFF020EE926000EEA22500E06
:101C5000EE6E020EED6E65C0E9FF66C0EAFF840E0F
:101C6000EF6E8751881107E005D088C0FAFF0001A8
:101C70008751F96EFADF0001849F020EE15C02E2F7
:101C8000E16AE552E16EE552E7CFD9FF1200D9CF04
:101C9000E6FFE1CFD9FFE65200017F8F040EE66E2A
:101CA000E66AE66A540EE66E0F0EE66E7AEC19F0FE
:101CB000146E050EE15E1450DF6ADF50146E156A73
:101CC000140E145C000E155810E2DF50040DF3CF13
:101CD000E9FFF4CFEAFF000EE926020EEA22EE6ADF
:101CE000EE6AEE6AEE6ADF2AE8D7648C010EE66ED1
:101CF000E66AE66A620EE66E000EE66E7AEC19F0AF
:101D0000146E050EE15E1450649C0001080E716FA4
:101D1000020E726F000E636F020E646F63C065F097
:101D200064C066F052C261F0615103E1100E606F51
:101D300012D0200E606F010EE66EE66A610EE66E4E
:101D4000000EE66E010EE66EE66AF3EC16F0146E17
:101D5000060EE15E1450E552E552E7CFD9FF1200BE
:101D6000D9CFE6FFE1CFD9FF020EE126000EDE6EED
:101D7000020EDD6EFD0EDB50E824166EFE0EDB500B
:101D8000040DF3501624040DF350146E156A020E60
:101D90000F0B05E0D89015321432E806FBE1D8901D
:101DA00014361536D89014361536D9CFE9FFDACF68
:101DB000EAFF1450EE261550ED22DECFE9FFDDCF0D
:101DC000EAFFEF9EFD0EDB500FE1FE0EEA6ADB3408
:101DD000FE0BEA36E96E670EE926000EEA22DECF38
:101DE000EEFFDDCFEDFF0ED0FE0EEA6ADB34FE0B18
:101DF000EA36E96E710EE926000EEA22DECFEEFF2A
:101E0000DDCFEDFFDECFE9FFDDCFEAFFEF9CDECFD8
:101E1000E9FFDDCFEAFF040EE926000EEA22EF8C8F
:101E2000020EE15C02E2E16AE552E16EE552E7CFC3
:101E3000D9FF1200D9CFE6FFE1CFD9FF020EE1268C
:101E4000FE0EDB50156A530F146E0F0E152214C0D0
:101E5000DEFF15C0DDFFDECFE9FFDDCFEAFFFD0EBF
:101E6000DBCFEFFFDBA407D0E66AFE0EDBCFE6FF99
:101E700077DFE552E552FD0EDBA208D0010EE66EDB
:101E8000FE0EDBCFE6FF6CDFE552E552020EE15CB1
:101E900002E2E16AE552E16EE552E7CFD9FF1200B6
:101EA000D9CFE6FFE1CFD9FF020EE126FE0EDB50CF
:101EB00020E165C0E9FF66C0EAFFEE52080EEF6E52
:101EC00065C0E9FF66C0EAFF020EE926000EEA22BD
:101ED000500EEE6E020EED6E65C0E9FF66C0EAFFC1
:101EE0008C0EEF6E71C0E9FF72C0EAFF840EEF6ED8
:101EF0003DD0FD0EDB50E824166EFE0EDB50040DC7
:101F0000F3501624040DF3CF14F0F4CF15F0000EA7
:101F10001426020E152214C0DEFF15C0DDFF840E4C
:101F2000146EDECFE9FFDDCFEAFF1450EF12FD0E95
:101F3000DB50E824166EFE0EDB50040DF350162421
:101F4000010F040DF3CF14F0F4CF15F0000E14269A
:101F5000020E152214C0DEFF15C0DDFF840E146EC4
:101F6000DECFE9FFDDCFEAFF1450EF12020EE15C95
:101F700002E2E16AE552E16EE552E7CFD9FF1200D5
:101F8000D9CFE6FFE1CFD9FF020EE126FD0EDB50EF
:101F90000FE0FE0EEA6ADB34FE0BEA36E96E710EE4
:101FA000E926000EEA22EECFDEFFEDCFDDFF0ED0F8
:101FB000FE0EEA6ADB34FE0BEA36E96E670EE926AE
:101FC000000EEA22EECFDEFFEDCFDDFFDECFE9FF30
:101FD000DDCFEAFF020EE926000EEA22FB0EDBCF80
:101FE000EEFFFC0EDBCFEDFFDECFE9FFDDCFEAFF3A
:101FF000EE52FA0EDBCFEFFF400E146EDECFE9FF9C
:10200000DDCFEAFF1450EF16880E146EDECFE9FF25
:10201000DDCFEAFF1450EF12FD0EDB500CE0FE0E98
:10202000EA6ADB34FE0BEA36E96E710EE926000E31
:10203000EA22EF740BD0FE0EEA6ADB34FE0BEA36BE
:10204000E96E670EE926000EEA22EF74DECF14F087
:10205000DDCF15F014C0F3FF15C0F4FF020EE15CF4
:1020600003E200D0E16AE552E16EE552E7CFD9FF25
:102070001200D9CFE6FFE1CFD9FF64A84ED0FE0E03
:10208000EA6ADB34FE0BEA36E96E710EE926000ED1
:10209000EA22EE50EFCFEAFFE96E400EEE16EE6A4E
:1020A000EE6AEE6AFE0EEA6ADB34FE0BEA36E96E91
:1020B000710EE926000EEA22EE50EFCFEAFFE96E3C
:1020C000EE7CFE0EEA6ADB34FE0BEA36E96E710E38
:1020D000E926000EEA22EF74400E146EFE0EEA6A44
:1020E000DB34FE0BEA36E96E710EE926000EEA22B9
:1020F000EE50EFCFEAFFE96E1450EF16FE0EEA6ADB
:10210000DB34FE0BEA36E96E710EE926000EEA2298
:10211000EE50EFCFEAFFE96EEF7CE552E7CFD9FF53
:022120001200AB
:0E212200DACFE4FFE2CFDAFFE652E552E5CF76
:10213000DAFF1100D8CFE4FFE0CFE4FFE46EDACF9E
:10214000E4FFE2CFDAFFE652E552E5CFDAFFE550F1
:10215000E5CFE0FFE5CFD8FF100005D866EC08F02A
:1021600088D8FCD712000F0EC11202D816EF08F063
:10217000D9CFE6FFE1CFD9FFE652010EDF6EF00EB8
:10218000936EB00E946E7E6A7F6AF19E7888788A2C
:10219000788C788E0001A66BA76BA86BA96BAA6BD5
:1021A000AB6BAC6BAD6B0001C26BC36BC46BC56B2F
:1021B00002016B6B6BC26AF26BC269F26E6B6EC22C
:1021C0006DF26EC26CF20201686B68C267F268C29F
:1021D00066F268C265F268C264F268C263F268C2FD
:1021E00062F268C261F282BE03D00001C16B1DD0F1
:1021F00082BA04D00001050EC16F17D081BE04D091
:102200000001020EC16F11D081BC04D00001030E89
:10221000C16F0BD081BA04D00001040EC16F05D08C
:1022200081B803D00001010EC16F630E0001C15DD2
:102230000FE1000EE66EE66A54EC19F0E552E55245
:102240000001C16FC151050802E2C16B01D0DF6A14
:10225000DF500AE0C1C0E6FF000EE66EE66A63ECFE
:1022600019F0E552E552E552E552E552E7CFD9FFC4
:102270001200200E0001E76E6019E8AE02D0E734CC
:1022800002D0E750605D03E36450020B01E01FD011
:102290000001C151050A18E0010A13E0070A0FE026
:1022A000010A0BE0030A07E0010A03E021EC16F043
:1022B0000ED00ED80CD007DB0AD060DB08D0BCDB18
:1022C00006D072EC15F003D0CAEC15F000D0120065
:1022D000D9CFE6FFE1CFD9FFE6528150400B01E0B4
:1022E000010E1D6E8150100B100A01E0010E1C6ED4
:1022F0008150200B200A01E0010E1C02F3501D0248
:10230000F350040DF3CF1BF08150100B01E0010ED0
:102310001A6E8150400B01E0010E196E8150200BA6
:10232000200A01E0010E1902F3501A02F350E824CA
:10233000186E0001CA0502E0000E01D0010E176EF2
:102340008150400B400A01E0010E1714166E8150B7
:10235000100B01E0010E156E8150200B01E0010E03
:10236000146E8150400B400A01E0010E1402F3503C
:102370001502F350161018241B2400019E6F000153
:10238000CA0502E0000E01D0010E176E8150400B0D
:1023900001E0010E166E8150100B01E0010E1610C7
:1023A0001710156E8150200B01E0010E146E815044
:1023B000400B01E0010E14101502F35035E082507D
:1023C000200B200A01E0010E146E156A14BE156878
:1023D00014500001B1271550B2238250800B800A9F
:1023E00001E0010E146E156A14BE15681450B15F39
:1023F0001550B25B8150800B800A01E0010E146E13
:10240000156A14BE15681450B3271550B4238250B2
:10241000100B100A01E0010E146E156A14BE156847
:102420001450B35F1550B45B8150200B01E0010ED6
:10243000166E0001CA5102E0000E01D0010E156EA9
:102440008150400B400A01E0010E146E8150100BC8
:10245000100A01E0010E1414151416142DE0825018
:10246000200B200A01E0010E030DF3CF16F081507E
:10247000800B800A01E0010E1624146E156A14BE4A
:10248000156814500001B55F1550B65B8250800B83
:10249000800A01E0010E030DF3CF16F08250100BFD
:1024A000100A01E0010E1624146E156A14BE156898
:1024B0001450B5271550B6230001BA51B219E8AE31
:1024C00002D0B23504D0B151B95DB251BA5905E26A
:1024D000B951B15FBA51B25B9F2B08680968B9C0A6
:1024E0000DF0BAC00EF027EC19F006C014F007C0CA
:1024F00015F00001B2511518E8AE02D0153404D021
:102500001450B15D1550B25905E2B951B127BA5115
:10251000B2239F07BC51B419E8AE02D0B43504D041
:10252000B351BB5DB451BC5905E2BB51B35FBC5163
:10253000B45BA02B08680968BBC00DF0BCC00EF0EE
:1025400027EC19F006C014F007C015F00001B451D3
:102550001518E8AE02D0153404D01450B35D1550F0
:10256000B45905E2BB51B327BC51B423A007BE51F7
:10257000B619E8AE02D0B63504D0B551BD5DB6513E
:10258000BE5909E2BD51B55FBE51B65BB80EBD6F15
:102590000B0EBE6FA12BBDC014F0BEC015F0146CA5
:1025A000151E000E1522B6511518E8AE02D01534CE
:1025B00004D01450B55D1550B65909E2BD51B52788
:1025C000BE51B623B80EBD6F0B0EBE6FA107000142
:1025D000C851C91102E0000E01D0010E176E8250E1
:1025E000800B01E0010E166E8250200B01E0010EFF
:1025F000156E8150800B01E0010E146E8250100B9D
:1026000001E0010E141415141614171416E0100E20
:10261000C81902E1270EC91902E0000E01D0010E0F
:10262000640E0001BD6FBE6B9F6BB16BB26BA06B94
:10263000B36BB46BA16BB56BB66B0001C851C9111C
:1026400003E0C807000EC95BC607000EC75BC65192
:10265000C71149E1640EC66FC76B8250200B200A78
:1026600001E0010E146E8250800B800A01E0010E21
:10267000141012E00F0E0001B95F000EBA5B500E8D
:10268000BAAF02D0D89003D0B95D000EBA5903E2B8
:10269000500EB96FBA6B05D00001F40EB96F010E80
:1026A000BA6F8150800B800A01E0010E146E8250D7
:1026B000100B100A01E0010E141011E00F0EBB5FA9
:1026C000000EBC5B500EBCAF02D0D89003D0BB5DF7
:1026D000000EBC5903E2500EBB6FBC6B04D0F40E6D
:1026E000BB6F010EBC6F81B833D08250200B200A23
:1026F00001E0010E176E8250800B800A01E0010E8E
:10270000166E8150800B800A01E0010E156E82501A
:10271000100B100A01E0010E152416241724146E64
:10272000010EE76E1418E8AE02D0143403D0E7505F
:10273000D880145407E2280E0001B96FBA6BBB6F42
:10274000BC6B06D01E0E0001B96FBA6BBB6FBC6BC1
:102750008250200B200A01E0010E166E8250800B81
:10276000800A01E0010E156E8150800B800A01E0A5
:10277000010E146E8250100B100A01E0010E1410AD
:10278000151016100001CB6F8150100B01E0010EE7
:10279000156E8150100B01E0010E146E8150400B3C
:1027A000400A01E0010E1414151406E0CC5104E1B6
:1027B000CB5102E0010ECA6FCBC0CCF081BCCA6B1A
:1027C0000001A651A71102E1000E08D0A6C0E9FF42
:1027D000A7C0EAFFEF50800B01E0010E00091EE1E7
:1027E0009EC06CF29FC06DF2A0C06EF2A1C06FF2ED
:1027F0009F6BA06BA16B040EE66E6C0EE66E020E74
:10280000E66E010EE66EE66EC0EC0FF0146E050E7D
:10281000E15E1450F3CFA6F0F4CFA7F00001AA5167
:10282000AB1102E1000E08D0AAC0E9FFABC0EAFF7D
:10283000EF50800B01E0010E000940E10201616BE5
:10284000636B8150200B200A01E0010E146E815051
:10285000400B400A01E0010E141416E082B804D0C7
:10286000010E616F1A0E636F81BE02D02A0E636F74
:1028700082BE04D0030E616F2B0E636F82BA04D048
:10288000010E616F2B0E636F626B646B656B666B21
:10289000676B686B080EE66E610EE66E020EE66E02
:1028A000010EE66E030EE66EC0EC0FF0146E050E20
:1028B000E15E1450F3CFAAF0F4CFABF0E552E5524D
:1028C000E7CFD9FF12000001AA51AB1102E1000EBF
:1028D00008D0AAC0E9FFABC0EAFFEF50800B01E0CF
:1028E000010E00094AE10201616B626B82B803D0FC
:1028F000520E636F08D08150800B800A01E0010EF8
:10290000510DF3CF63F282BE03D0500E646F08D036
:102910008250200B200A01E0010E4F0DF3CF64F22C
:102920008150400B400A01E0010E280DF3CF65F203
:102930008150200B200A01E0010EE10DF3CF66F279
:102940008150100B100A01E0010E2C0DF3CF67F23D
:10295000686B080EE66E610EE66E020EE66E010E04
:10296000E66E030EE66EC0EC0FF0146E050EE15E2F
:102970001450F3CFAAF0F4CFABF012000001A8512D
:10298000A91102E1000E08D0A8C0E9FFA9C0EAFF22
:10299000EF50800B01E0010E00094CE18150100B5B
:1029A000100A01E0010E040DF3CF15F08150200B49
:1029B000200A01E0010EE824146E8150400B400A09
:1029C00001E0010E142415240201696F8250200BCE
:1029D000200A01E0010E7F0DF3CF14F08250800B2E
:1029E00001E0010E800DF35014246A6F8150800BBA
:1029F000800A01E0010E7F0DF3CF14F08250100B1E
:102A000001E0010E800DF35014246B6F030EE66E8F
:102A1000690EE66E020EE66E010EE66E020EE66EC0
:102A2000C0EC0FF0146E050EE15E1450F3CFA8F069
:102A3000F4CFA9F000D012000001AA51AB1102E1BD
:102A4000000E08D0AAC0E9FFABC0EAFFEF50800B30
:102A500001E0010E000945E10201616B636B82B880
:102A600003D0616B420E636F81BE03D0616B410E78
:102A7000636F82BE04D0030E616F050E636F82BA6E
:102A800004D0030E616F090E636F81BC04D0010E88
:102A9000616F050E636F81BA04D0010E616F090E7C
:102AA000636F81B804D0010E616F130E636F626BA8
:102AB000646B656B666B676B686B080EE66E610E28
:102AC000E66E020EE66E010EE66E030EE66EC0ECDA
:102AD0000FF0146E050EE15E1450F3CFAAF0F4CFA0
:102AE000ABF012000001AA51AB1102E1000E08D0B8
:102AF000AAC0E9FFABC0EAFFEF50800B01E0010E76
:102B0000000947E10201616B636B82B804D00A0ED1
:102B1000616F180E636F81BE04D00A0E616F070EDD
:102B2000636F82BE04D00A0E616F050E636F82BAB6
:102B300004D00A0E616F090E636F81BC04D00A0EC7
:102B4000616F0C0E636F81BA04D00A0E616F160EAE
:102B5000636F81B804D00A0E616F2C0E636F626BD5
:102B6000646B656B666B676B686B080EE66E610E77
:102B7000E66E020EE66E010EE66E030EE66EC0EC29
:102B80000FF0146E050EE15E1450F3CFAAF0F4CFEF
:102B9000ABF012000001AA51AB1102E1000E08D007
:102BA000AAC0E9FFABC0EAFFEF50800B01E0010EC5
:102BB000000946E10201616B636B82B804D0010E2B
:102BC000616F3D0E636F81BE04D0010E616F1D0EFB
:102BD000636F82BE04D0030E616F2B0E636F82BAE7
:102BE00004D0010E616F2B0E636F81BC03D0080E01
:102BF000616F636F81BA04D0080E616F070E636F57
:102C000081B804D0040E616F3D0E636F626B646B1C
:102C1000656B666B676B686B080EE66E610EE66E41
:102C2000020EE66E010EE66E030EE66EC0EC0FF0CD
:102C3000146E050EE15E1450F3CFAAF0F4CFABF0A2
:102C40001200D9CFE6FFE1CFD9FF020EE126000145
:102C5000C251C31102E1000E08D0C2C0E9FFC3C0D7
:102C6000EAFFEF50800B01E0010E000901E07BD08C
:102C700002017851370A33E0B60A04E0010A01E0A4
:102C80005FD05ED0810EB86F81AE03D0010EB96FF8
:102C900001D0B96B0001C451C51102E1000E08D08A
:102CA000C4C0E9FFC5C0EAFFEF50800B01E0010E90
:102CB000000914E1400EE66EB80EE66E020EE66EF6
:102CC000010EE66E040EE66EC0EC0FF0146E050EFB
:102CD000E15E1450F3CFC4F0F4CFC5F031D0000161
:102CE000C451C51102E1000E08D0C4C0E9FFC5C03F
:102CF000EAFFEF50800B01E0010E000920E1020124
:102D0000370EB86F8250100B100A01E0010E500D03
:102D1000F3CFB9F2BA6B400EE66EB80EE66E020E55
:102D2000E66E010EE66E040EE66EC0EC0FF0146E59
:102D3000050EE15E1450F3CFC4F0F4CFC5F000D01F
:102D4000400EE66E780EE66E020EE66EE66A040E41
:102D5000E66EC0EC0FF0146E050EE15E1450F3CF7A
:102D6000C2F0F4CFC3F0020EE15C02E2E16AE55288
:102D7000E16EE552E7CFD9FF1200120012001200F7
:102D8000120019EF18F012001E0EE66E010EE66E2C
:102D90001AEC0FF0E552E5521E0EE66E020EE66EDC
:102DA0001AEC0FF0E552E5521E0EE66E030EE66ECB
:102DB0001AEC0FF0E552E5521E0EE66E040EE66EBA
:102DC0001AEC0FF0E552E552120064840001080E7F
:102DD000BF6F070EC06FBF07000EC05BBF51C011B1
:102DE000FAE164941200D9CFE6FFE1CFD9FFFD0EDE
:102DF000DBCF08F0FE0EDBCF09F0720E081801E100
:102E0000095033E0E868081802E17F0E09182BE04A
:102E1000740E081801E1095024E0750E081801E14C
:102E200009501DE0730E081801E1095016E0030E69
:102E3000081801E109500FE0020E081801E10950DD
:102E400008E0010E081801E1095001E010D09CDFF4
:102E50000FD099DF0DD095DF0BD091DF09D08DDF3A
:102E600007D08CDF05D08CDF03D0000001D000D06C
:0C2E7000010E00D0E552E7CFD9FF1200A0
:042E7C00120100023D
:102E800000000008EA220500010001020001090219
:102E90008200040100C032090400000103010200A5
:102EA00009211101000122340007058103040001FA
:102EB00009040100020300000009211101000122A0
:102EC00031000705820340000107050203400001AD
:102ED000090402000203010100092111010001227D
:102EE0003F000705830308000107050303080001ED
:102EF000090403000203000000092111010001225E
:102F00001D0007058403400001070504034000017C
:102F100005010902A1010901A100050919012903FF
:102F20001500250195037501810295017505810143
:102F300005010930093109381581257F7508950388
:102F40008106C0C005010905A10115002501350054
:102F500045017501950305091901290381029505AC
:102F6000810105010930093126FF0046FF0075087F
:102F700095028102C005010906A101050719E02992
:102F8000E7150025017501950881029501750881F5
:102F9000039505750105081901290591029501752B
:102FA0000391039506750815002565050719002985
:102FB000658100C00600FF0901A101190129401522
:102FC0000026FF00750895408100190129409100F5
:102FD000C004030904260342006900740020005461
:102FE00000720061006400650020004F006E006503
:102FF0000020004C00540044002E002E034D0069B8
:1030000000630072006F0020004D0075006C0074BA
:10301000006900200043006F006E00740072006FB2
:10302000006C006C00650072008E2ED12FD52FFB36
:013030002F70
:0E303200020150511F0B010801E0B8D0060E3C
:10304000515D01E077D05351230A73E0010A3AE061
:10305000030A01E06FD05451030A28E0010A1BE083
:10306000030A0EE0010A01E02CD00001A00E7D6FE2
:103070002E0E7E6F090E806F816BC00E7F6F21D088
:103080000001B90E7D6F2E0E7E6F090E806F816B71
:10309000C00E7F6F16D00001D90E7D6F2E0E7E6F91
:1030A000090E806F816BC00E7F6F0BD00001F90E8F
:1030B0007D6F2E0E7E6F090E806F816BC00E7F6F4D
:1030C00000D038D05451030A28E0010A1BE0030A5B
:1030D0000EE0010A01E02CD00001100E7D6F2F0ED2
:1030E0007E6F340E806F816BC00E7F6F21D0000128
:1030F000440E7D6F2F0E7E6F310E806F816BC00E80
:103100007F6F16D00001750E7D6F2F0E7E6F3F0E04
:10311000806F816BC00E7F6F0BD00001B40E7D6F8E
:103120002F0E7E6F1D0E806F816BC00E7F6F00D0E3
:1031300001D000D002015051600BE842E842E84261
:10314000E842E842010801E032D051510B0A29E07F
:10315000080A1CE0090A14E0080A07E00B0A04E068
:10316000080A01E024D023D022D00001D70E7D6FC1
:10317000000E7E6F010E806F816BC10E7F6F17D0C6
:103180000001800E7F6F53C2D7F011D00001D80E1E
:103190007D6F000E7E6F010E806F816B810E7F6FE1
:1031A00006D00001800E7F6F52C2D8F000D012000E
:1031B0001E0EF66E100EF76E000EF86E000109007E
:1031C000F550D26F0900F550D36F03E1D26701D0FB
:1031D0003DD00900F550CD6F0900F550CE6F0900C4
:1031E000F550CF6F09000900F550E96E0900F55060
:1031F000EA6E090009000900F550D06F0900F5508A
:10320000D16F09000900F6CFD4F0F7CFD5F0F8CF91
:10321000D6F0CDC0F6FFCEC0F7FFCFC0F8FF00015B
:10322000D05302E1D15307E00900F550EE6ED0070C
:10323000F8E2D107F9D7D4C0F6FFD5C0F7FFD6C062
:0E324000F8FF0001D207000ED35BBFD71200CB
:02324E0009C0B5
:1032500013F008C012F008500D02F4CF07F0F3CFBE
:1032600006F009500E02F4CF09F0F3CF08F00D027A
:10327000F3500726F4500822E86A092212500E0281
:10328000F3500726F4500822E86A09220EAE4DEFEB
:1032900019F01250085E1350095A13AE000C0D506D
:0832A000085E0E50095A000CF3
:0832A800D9CFE6FFE1CFD9FF09
:1032B000FD0EDB50A96EA66AA680A85000D0E5528C
:1032C000E7CFD9FF1200D9CFE6FFE1CFD9FFFD0E3E
:1032D000DB50A96EFC0EDB50A86E040EA66E550ED8
:1032E000A76EAA0EA76EA682A6B2FED7E552E7CFBA
:0432F000D9FF1200F0
:0C32F400FE0EE3CFE9FFFF0EE3CFEAFF80
:10330000E9CFF3FFEACFF4FFFB0EE35003E1FC0E3D
:10331000E35009E0FB0EE30602E2FC0EE306FD0EBD
:08332000E350EE6EF1D712003C
:08332800000EF36E00EE00F050
:10333000030E01D81200EA6002D0EE6AFCD7F35007
:08334000E9601200EE6AFCD7FF
:0833480011EE00F021EE00F08F
:10335000F86A019CD8EC18F003EC08F0ADEC10F022
:04336000FBD7120085
:0C33640063000000006400000000000096
:020000040030CA
:0100000000FF
:0100010032CC
:0100020001FC
:010003001EDE
:0100050000FA
:0100060001F8
:0100080003F4
:01000900C036
:01000A0003F2
:01000B00E014
:01000C0003F0
:01000D0040B2
:00000001FF
